:100000000208F1E308E3080000E42AE42A0000E320
:1000100008E3080000E100E420E1C8E3D010B600E6
:100020000A00001000A878A8780000AF8AAF8A0004
:1000300000A878A87800009FE0AF809FE0AF801014
:10004000B6000A0000FFA000000000029EE72702A1
:10005000CFE8D902E8E9A00302EA62031DEB1D0321
:1000600039EBD30356EC830375ED320393EDD003E4
:10007000B4EE7203CEEEEA03E8EF5C040BEFEC049F
:1000800030F07B0455F100047CF18204A4F1FF04FC
:10009000CEF27A04F9F2EF0526F3620555F3D105A5
:1000A00085F43B05B6F4A005EAF505061FF56406E0
:1000B00056F5C0068FF61A06CAF6700707F6C3078C
:1000C00046F7130788F76207F3F7D6083BF81E08D0
:1000D00085F86308D1F8A40920F8E40972F9220927
:1000E000C7F95E05050503050601050103010602C2
:1000F00005020302060305030303060405040304C3
:10010000062B2B0101010101010101010100205316
:100110006174656C6C6974652E32422D5220004208
:1001200075696C64202D2032312E30362E30360029
:100130005363616E6E696E672E2E2E005374657068
:10014000005363616E6E696E67204C6F7700536376
:10015000616E6E696E6720486967680042616E640F
:10016000204C6F77206C696D69740042616E642069
:1001700048696768206C696D6974004368616E6ED8
:10018000656C73005278204672657175656E63798F
:10019000005478204672657175656E6379005375F9
:1001A00062546F6E65202043682D457869740000A5
:1001B000000000000000000000001F1F1F1F0000C3
:1001C0000000000000000000000103010101000028
:1001D00000060902040F0000000F0102010F0000D9
:1001E0000003050F010100000006090909060000CF
:1001F0000006080E09060000000018181818000074
:1002000000001B1B1B1B00C0E0C006C00720050A26
:100210007E4B7F46B296DFFEDEF8E55A7004D2963A
:100220008002C296D007D006D0E022853C35853DBD
:1002300036AE4EBE000A2536F536E5F03535F535D5
:10024000C3E5459536E54495354008E5369543E5E3
:100250003595422275F0FF74FF800575F00074013A
:10026000755C20120207755800755900AF4EBF002B
:1002700002802CC0E0C0F075F006A4254CB4D20377
:10028000E48005B4FA0274CCF54C1206E5200603AE
:1002900012022BD0F0D0E040DA1206D10206BBC029
:1002A000F0854DF0A4D0F0C0E020060312022BD060
:1002B000E0401EC0E0C0F0253FF53FE5F0353EF5DB
:1002C0003ED0F0D0E0253DF53DE5F0353CF53C80F5
:1002D0001FE5F0B4000E85423E85423C85433F85D4
:1002E000433D800C85443E85443C85453F85453DE6
:1002F00022E53375F019A4F533C0F0E53275F01935
:10030000A485F034D0F025F0C0D0F532E53175F099
:1003100019A48534F0D0D035F0F5312285503585DB
:1003200051367B02C3E53633F536E53533F535DB3B
:10033000F3E55A42361205F230E408853C37853D34
:10034000388006853E37853F38E55A6004C296807E
:1003500002D296855A318537328538331202F1122E
:1003600005F230E40DC3E538954BF538E537954A8D
:0E037000F537C3E53833F538E53733F537E5B3
:10037E003633F536E53533F5357835E612046C0847
:10038E00B839F80000D2950000C295120722E55D3B
:10039E00B45305855D288003855C2875B074209262
:1003AE000875215475227880067521527522783091
:1003BE00070675214675226EE53EB53C07E53FB54D
:1003CE003D028003752652E5404541600375277452
:1003DE00E54E6015E54C75F006840475F00A84440C
:1003EE0030F524E5F04430F5257829760008B8314B
:1003FE00FAC37C1878337D08E633F618DDFADC2F65
:10040E00782D12045D8F2912045D8E2A8F2B120413
:10041E005D8E2C8F2D12045D8E2E8F30752F2E74C7
:10042E0080782112059EE61205BF08B831F82278B1
:10043E003012044E782F12044E782E12044E80B4D1
:10044E0074032630E301F674302630E701F622E617
:10045E00C4540F4430FEE6540F4430FF08227C088B
:10046E00C33392B000D2B100C2B1DCF5227C109041
:10047E00010E748012073890011F120734E4F55AEA
:10048E00900003FA7C067B011204D9900009FA7CD5
:10049E00067B261204D9E4755A02900025FA7C06D2
:1004AE007B011204D990002BFA7C067B261204D90C
:1004BE00755A0090000F7AEA7C167B011204D975EA
:1004CE005A029000317AEA7C167B01E4C004C0E047
:0D04DE0093F557EA1204F0D0E0040ADCF1B7
:1004EB00D004DBEA22C0E0C0E0120512E55A44A0BA
:1004FB00120528D0E0120528E55712052812058CA5
:10050B00D0E07D1A0205DA75B0FF00C2B7120551B3
:10051B00D2B7120551C2B0120551C2B7227D087570
:10052B00B07E331205514007C2B01205518005D27F
:10053B00B0120551D2B7120551DDE4120551C2B705
:10054B0012055175B0FF7F040205D7F5F0120512A5
:10055B00E55A44A0120528E5F0120528120512E50C
:10056B005A44A11205287D08C2B7120551D2B71201
:10057B00055120B003C38001D3C2B712055133DD3F
:10058B00E7C2B7120551C2B0120551D2B7120551CD
:10059B00D2B022C4C0E054EF44E0F5B00000C2B5C5
:1005AB001205DAD0E0C454EF44E0F5B00000C2B558
:1005BB00801D7420C4C0E044F0F5B00000C2B5D07B
:1005CB00E0C444F0F5B00000C2B57F14DFFE227E1C
:1005DB00371205D5DEFB227403F5B0C0E0D2B5D0DF
:1005EB00E0C2B57E0080EAE47DF7238DB000309247
:1005FB0001041DBDEFF47D28DDFE22E55AC0E07538
:10060B005A0074FE120556F55074FF120556F5513B
:10061B00D0E0F55A784F74FDC0E0120556F618D0AD
:10062B00E014B4EFF3AB4EBB000F7B06C0E012053A
:10063B0056F618D0E014DBF422E54C240580EB12BF
:10064B0005F264FF54F770F78085E54E701D74EA70
:10065B00853C571204F004853D571204F004853E87
:10066B00571204F004853F570204F074FA854C5777
:10067B000204F0E54E702C74EAC0E0120556F53C0E
:10068B00D0E004C0E0120556F53DD0E004C0E01206
:10069B000556F53ED0E004120556F53F7540007542
:1006AB0041002274FA120556F54C1206E51206D1DA
:1006BB00E54C04040404C0E0120556F540D0E004F8
:1006CB00120556F54122E54C0404C0E0120556F51F
:1006DB003ED0E004120556F53F22E54CC0E0120572
:1006EB0056F53CD0E004120556F53D22853C57E506
:1006FB004C1204F004853D571204F004853E57124A
:10070B0004F004853F571204F0048540571204F09F
:10071B00048541570204F07821762008B831FA227B
:10072B007C1074C012059E80157C1074C012059E3F
:10073B0074009360091205BFDC0122A380F27420C0
:10074B001205BFDCF92212025B12031C7B6012053F
:10075B00DA1205F24408B4FF051205DA801A120505
:10076B00D5DBEB12025B12031C7B0A1205DADBFBF7
:10077B001205F2B4FFED80E62212025412031C7B29
:10078B00601205DA1205F2B4FF051205DA801A12AF
:10079B0005D5DBED12025412031C7B0A1205DADBC2
:1007AB00FB1205F2B4FFED80E6227853900047E58B
:1007BB005293F6A308B857F722758921C28E758D0F
:1007CB00FF758BBCD294D28E30B6FDC28EC29474A0
:0C07DB00C012059EE58B7C0D755B00C311
:1007E70094C0403603541F6031FB941E40027B1DAA
:1007F700EBF55B13C0D0540F6013FB74C012059E5A
:1008070074081205BFDC04D0D0800CDBF3D0D050C5
:100817000674071205BF1CEC600774201205BFDCC5
:10082700F9E55B6026C3940E502B74CD12059EE547
:100837005B13C0D0540724321205BFD0D0500474C4
:100847002B800274201205BF0205BD74CD12059ED0
:100857001205BD80EEC0E074CD12059E74391205F5
:10086700BF74CE12059E9000E3D0E023C0E0931240
:1008770005BFD0E004930205BF79051205DAD9FB5D
:100887002275F0109001AF744012059E7400931208
:1008970005BFA3D5F0F622120655755A021205DADE
:1008A70074FF120556B2E1F55774FF1204F0755A3A
:1008B7000274FF1205565402F55A1206062274D224
:1008C7001208DC402274D81208DC401B74DE1208C0
:1008D700DC401474E4F557120556B53C0BE5570494
:1008E700120556B53D02D322C322C2AF75815E758C
:1008F70090FF75B0FF1205E21205E21205E27402DD
:100907001205E4742812059E740C12059E742812B1
:10091700059E740112059E755A0274FF120556F55D
:10092700F054F0B4A0061205F220E70312047B7519
:10093700815ED297C207C206C205755A0274FF12BA
:1009470005565402F55A120606755C20755D20752A
:10095700F0489001BF12088E12072BD297755800E6
:1009670075590012031CE558B4FF1D1207C4120580
:0A097700F230E01630E11630E2160F
:1009810030E41630E51530E61530E71580DE8014C9
:10099100020A1D020A52020B3F8020020A87020A44
:1009A100F7020BA6E5592401F559E5583400F5582D
:1009B100B401067558FF12065580B6E55DB45303C0
:1009C10012089E12088812031C9001031207347545
:1009D1008911C29775B074E5406014B293C28E85D7
:1009E100408D85418BD28E209225108FEE80FB7534
:1009F100B077209214B293C28E758DFF758B15D28C
:100A01008E209205108FEE80FB75B0743092E0D28B
:100A110097E55DB4530312089E02095612025B1258
:100A2100031C7B901205DA1205F24408B4FF06128A
:100A310005DA0209561205D5DBEA12025B12031C24
:100A41007B301205DADBFB1205F24408B4FFEB80C0
:100A5100E412025412031C7B901205DA1205F244CF
:100A610008B4FF061205DA0209561205D5DBEA12AF
:100A7100025412031C7B301205DADBFB1205F2442F
:100A810008B4FFEB80E41202071206557F327E00A4
:100A91001EDE051FDFF880251205F264FF54F77092
:100AA100EF12064A1205DA755C20E54EB2E0F54E0A
:100AB100F55774FC1204F012067E020956E54E60E9
:100AC100E0E55DB4200EE55CB4720F755C201206A2
:100AD1007E12031C12064A020956755C72AE3EAFC5
:100AE1003C8F3E8E3CAE3FAF3D8F3F8E3D12031C8F
:100AF10012064A0209567F327E001EDE051FDFF80C
:100B010080261205F264FF54F770EF120655755AEC
:100B1100021205DA74FF120556B2E1F55774FF129D
:100B210004F012064A020936E55DB42005755D53ED
:100B31008003755D2012031C12064A020956120237
:060B410007D20512064A6E
:100B47009001301207347AFF12025B1205F2FB5450
:100B5700F7B4F740C3E549953DE548953C40E9E5DD
:100B67003D9547E53C954640DF1208C540DA12033C
:100B77001C791E1205DA1205DA1205F2FB54F7B4D6
:100B8700F712EB30E304D9EB80AE1207C41205DA93
:100B9700DADF80ACC20512020712064A02095612B2
:100BA700072B120655D207E4F54E12031C12064A0C
:100BB7001205F230E01D30E11A30E21930E4183046
:100BC700E50B30E60B30E70280E6020FB2020CCEEF
:100BD700020F128005804D020FB212064AE54D75CD
:100BE700F019A475310085F032F53312039990019D
:100BF7003C1207341205F230E00830E10F30E716F7
:100C070080F2120207E54D04F54D80CE120207E58A
:100C17004D14F54D80C474FB854D571204F0120234
:100C270007020FB285463C85463E85473D85473FCF
:100C3700C20512020712064A12031C90014112074D
:100C4700341205F230E00830E11030E71880F21274
:100C57000751853C46853D4780DB120784853C4626
:100C6700853D4780D085483C85483E85493D854937
:100C77003F12020712064A12031C90014E12073454
:100C87001205F230E00830E11030E71880F2120761
:100C970051853C48853D4980DB120784853C488562
:100CA7003D4980D074F48546571204F004854757B0
:100CB7001204F0048548571204F0048549571204BA
:100CC700F0120207020FB2120207D206E4F54C0433
:100CD700F54E90017B1207341206E51206D1120673
:100CE700BB12031C12064A1205F230E00830E11469
:100CF70030E72180EF120207E54C2406B4EA01E44D
:0B0D0700F54C80CE120207E54C94066C
:100D1200B4FA0274E4F54C80BE1202079001841208
:100D2200073412031C12064A1205F230E00B30E1BE
:100D32004C30E70280EF020DC8E53D2401F53DF598
:100D42003FE53C3400F53CF53E12031C1202077CE1
:100D52001E1205F220E0C5120880DCF5E53D2401F3
:100D6200F53DF53FE53C3400F53CF53E12031C121F
:100D720002071205F220E0A412088080DFC3E53DDD
:100D82009401F53DF53FE53C9400F53CF53E120338
:100D92001C1202077C1E1205F220E127120880DCD9
:100DA200F5C3E53D9401F53DF53FE53C9400F53C86
:100DB200F53E12031C1202071205F220E105120889
:100DC2008080DE020D1E900191120734E53C853EC3
:100DD2003CF53EE53D853F3DF53F12031C120207FF
:100DE20012064A1205F230E00A30E14330E702808F
:100DF200EF807DE53D2401F53DE53C3400F53C12F4
:100E0200031C1202077C1E1205F220E0D312088096
:100E1200DCF5E53D2401F53DE53C3400F53C1203EB
:100E22001C1202071205F220E0B612088080E3C30A
:100E3200E53D9401F53DE53C9400F53C12031C129E
:100E420002077C1E1205F220E123120880DCF5C3A2
:100E5200E53D9401F53DE53C9400F53C12031C127E
:100E620002071205F220E10512088080E2020DE27B
:100E7200E53C853E3CF53EE53D853F3DF53F900135
:100E82009E1207347552009000477853E55293F64C
:100E9200A308B857F7E540C395557007E541C395D8
:100EA20056600FE5522404F552B59CDB75520012D0
:0B0EB20002071207B5753100855332AE
:100EBD0085543385554085564112039912064A12C1
:100ECD0005F230E00B30E11730E53130E72280ECF0
:100EDD00120207E5522404B49C01E4F55280C812B5
:100EED000207C3E5529404B4FC027498F55280B71E
:100EFD001206F712020712064A020CD91206F71251
:100F0D000207020FB2D20685423C85423E85433D23
:100F1D0085433F12020712064A12031C90015C1210
:100F2D0007341205F230E00830E11030E71880F296
:100F3D00120751853C42853D4380DB120784853C79
:100F4D0042853D4380D085443C85443E85453D8565
:100F5D00453F12020712064A12031C90016B12073D
:100F6D00341205F230E00830E11030E71880F2124B
:100F7D000751853C44853D4580DB120784853C4403
:100F8D00853D4580D074F08542571204F0048543A9
:100F9D00571204F0048544571204F0048545571286
:0E0FAD0004F012020712064A1205DA02093693
:00000001FF
